:100000000C94D3020C9417030C9417030C9417034D
:100010000C9417030C9417030C9417030C941703F8
:100020000C9417030C9417030C94DA0D0C94AC0E7B
:100030000C9417030C9417030C9417030C941703D8
:100040000C9417030C94B6220C9417030C9417030A
:100050000C9417030C94491C0C9417030C9417036D
:100060000C9417030C9417030C9417030C941703A8
:100070000C9417030C9417030C9417030C94170398
:100080000C9417030C9417030C9417030C94170388
:100090000C9417030C9417030C9417030C94170378
:1000A0000C9417030C9417030C941703190F3B0FB0
:1000B00029103B0F2910800FA30F2910F80F0B10E8
:1000C000DA12DA12091309133F135F139014901414
:1000D0006A1390141A141A148114901490148A1428
:1000E0002714271427142714271427142714271438
:1000F0002714271427142714271427142714271428
:10010000391446144D1454145E14750A01E2012C7E
:10011000022C02E2746401160216010402040109B1
:1001200002090104020401150215010C020C012848
:10013000022800750A01E2012C022C02E27464011B
:10014000170217010802080115021501100210011B
:100150000C020C0111021101040204010F020F0133
:1001600028022800750A01E2012C022C02E27464C4
:100170000105020501050205010802080107020741
:10018000010C020C011702170128022800750A0150
:10019000E30116021602E301E3012B022B02E30145
:1001A000E30115021502E300750A01E301160216C8
:1001B00002E301E3012B022B02E3000000F0A12E79
:1001C000004C002A00E100E00000001E00140004C2
:1001D000001D00E200E2001F001A0016001B00E3F1
:1001E000002A00200008000700060050002C002113
:1001F000001500090019004F004B00220017000AEB
:1002000000050000003500015401520000E3000029
:10021000003400015401520000E3000000290023D3
:10022000001C000B00110000002A00240018000D23
:1002300000100052004E0025000C000E0036005148
:10024000002800260012000F0037002F002B002787
:10025000001300334238713000E0002D00310034CB
:1002600078E5002C00000001000100010001000100
:100270000000003A002F0036020100010001003B9F
:1002800000300037020100010001003C002F02266F
:10029000020100010001003D0030022702010001BF
:1002A0000001003E003402340001000000010001A2
:1002B0000001000000010000000100010001000039
:1002C000000100000001003F0038002D0024020062
:1002D0000001004000240021001E0027004A0041C8
:1002E00000250022001F00370001004200260023E5
:1002F00000200050000100430025022E022E004F76
:10030000004D004400450001000100010000000113
:10031000000100010001000100000069000100016E
:10032000000100010001006A000100043001000129
:1003300000010001004B004E00010001000100011E
:100340000001300100010001004A000100033001FA
:100350000002300000010001000100000001000067
:100360000001001408010000000100000001001A53
:100370000830082F082C0200000100350A520C50EA
:10038000002C00A9000100350852005100AC00AA61
:100390000019080100510C4F00AB00A8000608012D
:1003A0000001000100010001001B08A5000100AED2
:1003B0000001000100000016034500720067006F95
:1003C0000044006F007800200045005A000000162D
:1003D000034500720067006F0044006F0078002042
:1003E0000045005A0000000403090409026D0004DE
:1003F0000100A0FA09040000010301010009211114
:10040000010001223F000705810308000A090401D9
:10041000000103010200092111010001224D000722
:1004200005820308000A0904020001030000000914
:1004300021110100012236000705830308000A0983
:100440000403000103000000092111010001223909
:1004500000070584031000011201100100000008CC
:10046000EDFE071301000102000105010906A101CB
:10047000050719E029E71500250195087501810296
:100480000508190129059505750191029501750366
:100490009101050719002977150025019578750147
:1004A0008102C005010980A101850216010026B75D
:1004B000001A01002AB700751095018100C0050CD3
:1004C0000901A1018503160100269C021A01002AD8
:1004D0009C02751095018100C005010902A1010966
:1004E00001A10005091901290515002501950575CA
:1004F000018102950175038101050109300931155A
:1005000081257F95027508810609381581257F951B
:100510000175088106050C0A38021581257F9501B1
:1005200075088106C0C005010906A101050719E08B
:1005300029E71500250195087501810295017508C7
:10054000810105081901290595057501910295019B
:10055000750391010507190029FF150025FF950670
:1005600075088100C00000000000000000000000CD
:10057000010204060A0F17202C3A4A5D71879DB3C9
:10058000C7DAE9F5FCFFFCF5E9DAC7B39D87715DD1
:100590004A3A2C20170F0A0604020100000000004E
:1005A00000000000000011241FBECFEFDAE0DEBF24
:1005B000CDBF04B603FE24C08091FB019091FC01E5
:1005C000A091FD01B091FE018730904BA740B04B48
:1005D000B9F41092FB011092FC011092FD011092EF
:1005E000FE0114BE84B7877F84BF88E10FB6F894FC
:1005F00080936000109260000FBEE0E0FFE3099579
:1006000011E0A0E0B1E0EAEFF8E402C005900D923D
:10061000A433B107D9F711E0A4E3B1E001C01D9202
:10062000AB3FB107E1F70E941E0B0C947B240C94A6
:1006300000001092B9008AE08093B800089594EA0F
:100640009093BC009091BC0097FFFCCF9091B900B3
:10065000987F983021F0903111F081E008958093D7
:10066000BB0084E88093BC008091BC0087FFFCCF76
:100670008091B900887F883111F0803471F780E073
:10068000089584E98093BC008091BC0084FDFCCF78
:1006900008958093BB0084E88093BC008091BC00E7
:1006A00087FFFCCF9091B900987F81E0983209F4E0
:1006B00080E0089584E88093BC008091BC0087FFAF
:1006C000FCCF8091BB00089580910101811115C07C
:1006D00080E40E941F038093010181110CC082E11C
:1006E0000E94490380930101811105C08FEF0E9490
:1006F0004903809301010E94410384B1807F84B942
:1007000085B1807F85B98AB1837F8AB98BB1837FB8
:100710008BB93E98469808950E941F058093010169
:100720000E94640380B38C7080BB81B3836F81BBF4
:10073000A5E3B1E0E3E4F1E08EE08E0F11921D92AB
:100740008E13FCCF0C940905BF92CF92DF92EF92EB
:10075000FF920F931F93CF93DF9380910101882322
:1007600079F0809134018F5F80933401811108C04A
:100770000E941F0580930101811102C00E94B104F3
:1007800005E311E0C0E0D0E0DD24D39482E0C82E80
:10079000EE24E394F12CC730D10500F580910101DE
:1007A000811164C080E40E941F03809301018111C4
:1007B00012C082E10E9449038093010181110BC0A4
:1007C000C7010C2E01C0880F0A94EAF780950E9499
:1007D0004903809301010E94410348C0CA30A1F03F
:1007E00028F4C83059F0C93061F005C0CC3089F028
:1007F00070F0CD3089F0209A289810C0219A29985D
:100800000DC0229A2A980AC0239A2B9807C0529AA0
:1008100001C0539A5B9802C03E9A469890EA9A9516
:10082000F1F79FB1799902C082E001C080E0917038
:100830009D25982B7C9902C084E001C080E0892B23
:100840007D9902C038E001C030E0832B7E9902C060
:1008500020E101C020E0822B9FB19095991F99273C
:10086000991F9295990F907E892B0FC0809101015D
:10087000811149C080E40E941F03809301018823F5
:1008800079F1B12C0E9441038B2DF80190819817CA
:1008900019F08083C09200010E94640321960F5FCB
:1008A0001F4FCE30D10509F076CF8091000188230B
:1008B00061F1815080930001882339F08FE99FE036
:1008C0000197F1F700C0000020C0A3E4B1E0E5E328
:1008D000F1E0CF01825F91919D938E13FCCF15C003
:1008E00083E10E944903809301018111CACF81E411
:1008F0000E941F03809301018111C3CF0E945A03FC
:10090000B82EB094BFCF80E0C0CF0E94AF0481E08A
:10091000DF91CF911F910F91FF90EF90DF90CF90DB
:10092000BF900895E82FF0E0ED5BFE4F80810895C1
:1009300008950F931F93CF93DF93C3E4D1E010E0AA
:100940000C2F025F899190E00E946F1B180F0C130F
:10095000F9CF812FDF91CF911F910F9108950C94C2
:100960009E0556985E9825982D9826982E9827983B
:100970002F988FEF90E09093890080938800909358
:100980008B0080938A0090938D0080938C00259A31
:100990002D9A2FEF80E792E0215080409040E1F7C0
:1009A00000C00000269A2E9A2FEF80E792E0215097
:1009B00080409040E1F700C00000279A2F9A2FEF67
:1009C00080E792E0215080409040E1F700C00000B5
:1009D00025982D982FEF80E792E02150804090409D
:1009E000E1F700C0000026982E982FEF80E792E0F4
:1009F000215080409040E1F700C0000027982F98D8
:100A000056985E9825982D9826982E9827982F9876
:100A1000089589EA8093800089E08093810024987A
:100A20002C983F988AB18F748AB96E98479A8BB187
:100A3000806B8BB9769A0E94B1040C949D0580E27C
:100A4000809301018091510181110EC00E94190310
:100A500081E0809351012FEF83ED90E3215080409E
:100A60009040E1F700C0000080E40E941F038093E3
:100A7000010181112EC00E9449038093010181115F
:100A800028C00E94490380930101811122C08FE395
:100A90000E9449038093010181111BC00E94410300
:100AA00080E40E941F0380930101811112C08CE039
:100AB0000E9449038093010181110BC00E944903E8
:100AC00080930101811105C08FE30E944903809347
:100AD00001010E944103809101010895FC016230EF
:100AE000B9F028F4662341F0613061F023C063302F
:100AF000A9F06430C9F01EC082818823D9F088EA49
:100B000091E0089582818823A9F08DE891E008950D
:100B10008281882379F084E691E008958281882398
:100B200049F083E391E008958281882319F08AE0F7
:100B300091E0089580E090E0089508956091BD01EE
:100B40007091BE018091BF019091C0010E947B1BFA
:100B500056985E9825982D9826982E9827982F9825
:100B6000813019F0823021F00895259A2D9A089548
:100B7000269A2E9A089581E0089581E008950C94B4
:100B8000BD0508950F931F93CF93DF938C01FC0154
:100B9000C081D181CE010E94F419BE010E946B0672
:100BA000EC01B8010E94BF05882309F48DC0F8014B
:100BB0008281882309F44AC080915D0181111FC0A0
:100BC000C431F0E5DF0709F051C00E94C10581E0A2
:100BD00080935D010E94131C90935C0180935B01E4
:100BE0001092540110925601109255011092580122
:100BF0001092570110925A011092590165C08091CC
:100C00005B0190915C010E941F1C883C910570F46F
:100C100080915401E82FF0E0EE0FFF1FEB5AFE4FDA
:100C2000D183C0838F5F809354014EC0C43880E568
:100C3000D80721F0C538D04501F13AC0F8018281CA
:100C4000882341F01092520182E01EC0C438E0E5D2
:100C5000DE0759F580915201811106C086E20E949B
:100C60007E1186E20E94461282E01CC0C438F0E584
:100C7000DF0741F3C538D045D9F4F80182818823D4
:100C800031F01092530180E20E9495121DC08091B4
:100C90005301811106C087E20E947E1187E20E9403
:100CA000461280E20E949C120FC0C538D04529F33D
:100CB00081E08093520180935301C801DF91CF916D
:100CC0001F910F910C94BB0580E0DF91CF911F9194
:100CD0000F910895089596E0799FF001112494E50D
:100CE000899FE00DF11D1124E60FF11DEE0FFF1F8E
:100CF000E154FE4F859194910895880F991FFC014E
:100D0000E55CFF4F859194910895880F991FFC0130
:100D1000E554FE4F8591949108950F931F93CF93BF
:100D2000DF93EC01811520E3920750F5C11580E2B5
:100D3000D80708F0C3C0CB3BD10590F4C83AD10521
:100D400008F06AC0C53AD10508F05BC0C430D105CF
:100D500008F0D0C1219709F0CAC101E010E00AC231
:100D6000CF3FD10511F008F0C5C1C03FD10508F053
:100D7000A2C0CE01805E9109089708F4BBC1B7C13B
:100D8000C13090E5D90709F4A2C020F5C0318FE445
:100D9000D80770F4C11590E4D90708F094C0C115C4
:100DA00021E3D20708F0A3C1DD278E01106CE2C158
:100DB000C115D04509F09BC10E94FB148FEF94E34D
:100DC0002CE0815090402040E1F700C000000E94DC
:100DD0006E1CD0C1C11597E5D90758F4C03121E583
:100DE000D20708F01CC1C43180E5D80708F475C0EB
:100DF0007EC1CE0190578115904108F078C1DF7017
:100E000073C1C53AD10509F477C1C63AD10509F0D5
:100E100076C102E810E4AEC1C83AD10509F472C146
:100E2000C93AD10509F471C1CA3AD10509F470C1B2
:100E3000CB3AD10509F46FC1CC3AD10509F46EC1A2
:100E4000CD3AD10509F46DC1C03BD10509F46CC19F
:100E5000CE3AD10509F46BC1CF3AD10509F46AC184
:100E6000C13BD10509F469C1C23BD10509F468C190
:100E7000C33BD10509F467C1C43BD10509F466C180
:100E8000C53BD10509F465C1C63BD10509F464C170
:100E9000C73BD10509F463C1C83BD10509F462C160
:100EA000C93BD10509F461C1CA3BD10509F460C150
:100EB00000E014E45FC18E0110655CC1CE019F703B
:100EC0000E94850658C1DF708E01106A53C180915F
:100ED000DA0181608093DA014DC10E94131E8111F5
:100EE00002C00E94F91D0E94301E90E09093FB0109
:100EF0008093FA01C23080E5D80721F48091FA018D
:100F0000816086C0C43090E5D90721F48091FA0150
:100F100082607EC0C63020E5D20721F48091FA01BC
:100F2000846076C0C83080E5D80719F48091FA0152
:100F300027C0CA3090E5D90721F48091FA01806179
:100F400067C0CC3020E5D20721F48091FA0180629D
:100F50005FC0CE3080E5D80721F48091FA0180642B
:100F600057C0C03190E5D90721F48091FA0180681B
:100F70004FC0C23120E5D20729F48091FA01846084
:100F8000886046C0C33080E5D80721F48091FA011B
:100F90008E7F3EC0C53090E5D90721F48091FA01DB
:100FA0008D7F36C0C73020E5D20721F48091FA0149
:100FB0008B7F2EC0C93080E5D80719F48091FA01E3
:100FC00026C0CB3090E5D90721F48091FA018F7EBD
:100FD0001FC0CD3020E5D20721F48091FA018F7D2A
:100FE00017C0CF3080E5D80721F48091FA018F7BBC
:100FF0000FC0C13190E5D90721F48091FA018F77B4
:1010000007C0C331D04531F48091FA018B7F877FCF
:101010008093FA018091FA010E94341EABC08D2F9B
:1010200099278F70992781309105D9F49E012370FB
:10103000332702C0880F991F2A95E2F79C688E011A
:1010400044E0000F111F4A95E1F700271370802B31
:10105000912B53E0CC0FDD1F5A95E1F7C076DD27C9
:101060002FC08230910531F4DC2FCC278E01016F27
:10107000106A80C08330910569F4CE01837099278E
:1010800001E010E002C0000F111F8A95E2F7C801CD
:101090009C680FC084309105B9F4CE018370992704
:1010A00001E010E002C0000F111F8A95E2F7C801AD
:1010B0009A6823E0CC0FDD1F2A95E1F7C07ED77038
:1010C0008C010C2B1D2B56C08530910531F4DC2F83
:1010D000CC278E01046F106A4DC0069709F04AC0F4
:1010E000CF71DD27DC2FCC278E01106243C000E0DA
:1010F00010E040C08E013EC001E810E43BC003E8B0
:1011000010E438C002EE14E435C009EE14E432C035
:101110000AEE14E42FC005EB14E42CC006EB14E433
:1011200029C007EB14E426C00CEC14E423C00DEC3A
:1011300014E420C003E815E41DC00AE815E41AC051
:1011400002E915E417C004E915E414C001E216E44D
:1011500011C003E216E40EC004E216E40BC005E27F
:1011600016E408C006E216E405C007E216E402C071
:101170000AE216E4C801DF91CF911F910F91089503
:1011800096E0799FF001112494E5899FE00DF11D0F
:101190001124E60FF11DEE0FFF1FE154FE4F859164
:1011A0009491803E9105E0F4803C910558F581339F
:1011B000910509F46FC048F48932910509F463C0C0
:1011C0008A32910509F46DC072C089339105E9F046
:1011D00082389105D1F08533910509F44DC067C07F
:1011E000833E910581F138F4803E9105B9F0823E4D
:1011F0009105D9F05CC0863E910561F1873E91056D
:10120000A1F155C00E947D0608952091FA0120FDAC
:1012100002C021FF4CC080EE90E049C08091FA01ED
:1012200080FFF9CF89E390E042C08091FA0182FF0C
:101230000EC08091FA0184FF03C080E090E037C0C7
:1012400083EE90E034C08091FA0182FFF2CF82EE0B
:1012500090E02DC08091FA0183FF0BC08091FA01CC
:1012600084FDEBCF87EE90E022C08091FA0183FFEE
:10127000F5CF86EE90E01BC08091FA0185FF07C094
:1012800089E290E014C08091FA0185FFF9CF85E3EF
:1012900090E00DC08091FA0186FF07C08AE290E0DD
:1012A00006C08091FA0186FFF9CF81E390E00E94A9
:1012B0008D06089508950C945A0980916E01089541
:1012C000CF93DF9300D01F92CDB7DEB79C01809102
:1012D000F101843019F593E099833B832A8390933D
:1012E000E9008FEF9091E800815095FD06C095EDE3
:1012F0009A95F1F700008111F5CF8091E80085FF04
:101300000DC040E050E063E070E0CE0101960E9425
:10131000CA0B8091E8008E778093E8000F900F90C1
:101320000F90DF91CF910895CF93DF9300D01F925C
:10133000CDB7DEB72091F101243021F522E02983D9
:101340009B838A8383E08093E9008FEF9091E8008C
:10135000815095FD06C095ED9A95F1F70000811139
:10136000F5CF8091E80085FF0DC040E050E063E0DC
:1013700070E0CE0101960E94CA0B8091E8008E7742
:101380008093E8000F900F900F90DF91CF91089518
:101390002091F1012430F1F422E02093E9002FEFB5
:1013A0003091E800215035FD06C035ED3A95F1F752
:1013B00000002111F5CF2091E80025FF0BC040E08F
:1013C00050E065E070E00E94CA0B8091E8008E77E3
:1013D0008093E8000895CF93DF93EC019091F101A1
:1013E000943009F046C080910C018823D9F0809197
:1013F0000D018823B9F09093E9008FEF9091E800F8
:10140000815095FD06C095E19A95F1F70000811194
:10141000F5CF8091E80085FF2CC040E050E060E10E
:1014200070E017C081E08093E9008FEF9091E800B1
:10143000815095FD06C095ED9A95F1F70000811158
:10144000F5CF8091E80085FF14C040E050E068E0EF
:1014500070E0CE010E94CA0B8091E8008E778093E5
:10146000E80080E1FE01AEE5B1E001900D928A95C1
:10147000E1F7DF91CF9108958091F001811109C0CA
:101480000E945F0D0E94BC0D8091E20084608093F9
:10149000E20008951092F001089508950C94A3229B
:1014A0000E94041C0E94A9220E9462100C945B09F5
:1014B00042E061EC81E00E94D90C42E061EC82E004
:1014C0000E94D90C42E061EC83E00E94D90C42E119
:1014D00061EC84E00C94D90C8091F301833009F421
:1014E00055C030F4813071F0823009F48EC0089517
:1014F0008A3009F47AC08B3009F460C0893009F071
:101500009CC020C08091F201813A09F096C0809180
:10151000E800877F8093E8008091F6019091F701C1
:10152000892B21F460E18EE591E003C060E080E06A
:1015300090E070E00E94150C8091E8008B7780931A
:10154000E80008958091F201813209F076C080911F
:10155000F6019091F701009719F0039709F06DC01B
:101560008091E800877F8093E8008091E80082FD09
:1015700005C08091F1018111F8CF5FC08091F10029
:1015800080936E018091E8008B7753C08091F201C7
:10159000813A09F052C08091F6019091F701892BB0
:1015A00009F04BC08091E800877F8093E80080912C
:1015B000E80080FFFCCF80910C0136C08091F201E1
:1015C0008132D9F58091F6019091F701892BA9F527
:1015D0008091E800877F8093E8000E940E0D809143
:1015E000F40180930C010C94FB148091F201813280
:1015F00021F58091E800877F8093E8000E940E0D1E
:101600008091F50180936F0108958091F201813AF4
:10161000A1F48091E800877F8093E8008091E80042
:1016200080FFFCCF80916F018093F1008091E800F2
:101630008E778093E8000C940E0D089584B7877F11
:1016400084BF88E10FB6F894809360001092600028
:101650000FBE90E080E80FB6F894809361009093FD
:1016600061000FBE0E94B1100E945F0D0E94BC0D70
:101670008091E20084608093E20078940E9442109E
:101680000E94B31082E091E00E945D100E949122BE
:101690008091F101853069F40E94CB1B8091EF01AC
:1016A0008823B1F30E94F61B882391F30E94B40BA8
:1016B000EFCF0E94B910ECCF292F3327233031050B
:1016C000C9F064F42130310581F02230310509F090
:1016D00043C08DE690E02BEE33E042C0213231056D
:1016E000F1F02232310541F137C082E190E028E586
:1016F00034E036C099278130910541F08230910560
:1017000041F0892B49F5E7EEF3E005C0EFECF3E09B
:1017100002C0E7EBF3E0849190E09F0121C06430C8
:10172000D8F4E62FF0E0EE0FFF1FEE5DFE4F2081B4
:10173000318189E090E014C0643070F470E0FB0106
:10174000EE0FFF1FE65EFE4F20813181FB01EA5E56
:10175000FE4F808190E004C080E090E020E030E027
:10176000FA0131832083089580E189BD82E189BD3A
:1017700009B400FEFDCF8091D8008F7D8093D80002
:101780008091E00082608093E0008091E00081FD24
:10179000FCCF0895CF92DF92EF92FF920F931F93A9
:1017A000CF93DF93EC018B016A010E942D0D811113
:1017B00033C0C114D10439F0F60180819181081B36
:1017C000190BC80FD91FE12CF12C0115110519F1C6
:1017D0008091E80085FD16C08091E8008E778093A7
:1017E000E800C114D10449F0F60180819181E80E2E
:1017F000F91EF182E08285E00FC00E942D0D882342
:1018000021F30AC089918093F10001501109FFEF83
:10181000EF1AFF0ADACF80E0DF91CF911F910F918D
:10182000FF90EF90DF90CF9008952091F8013091D4
:10183000F9012617370748F06115710539F4209131
:10184000E8002E772093E80001C0B90140E061155F
:101850007105A9F12091F101222309F443C025303B
:1018600009F442C02091E80023FD40C02091E80027
:1018700022FD32C02091E80020FFE9CF4091F30023
:101880002091F20030E0342BFC01CF01611571058D
:1018900059F02830310540F481918093F100615076
:1018A00071092F5F3F4FF1CF41E02830310509F03A
:1018B00040E02091E8002E772093E800C8CF411146
:1018C000C9CF0AC08091F101882361F0853061F0B1
:1018D0008091E80083FD0AC08091E80082FFF2CF8A
:1018E00080E0089582E0089583E0089581E00895FE
:1018F0002091F8013091F9012617370748F061155A
:10190000710539F42091E8002E772093E80001C09A
:10191000B901FC0120E06115710591F18091F1019F
:10192000882309F440C0853009F43FC08091E80065
:1019300083FD3DC08091E80082FD2FC08091E800CA
:1019400080FFE9CF2091F3008091F20090E0922B8C
:101950006115710559F08830910540F42491209368
:10196000F1003196615071090196F2CF21E008979C
:1019700009F020E08091E8008E778093E800CBCFDB
:101980002111CCCF0AC08091F101882361F085300C
:1019900061F08091E80083FD0AC08091E80082FF39
:1019A000F2CF80E0089582E0089583E0089581E019
:1019B0000895982F973058F59093E900981739F0CB
:1019C0007091EC002091ED005091F00003C0242FA5
:1019D000762F50E021FF19C03091EB003E7F30930D
:1019E000EB003091ED003D7F3093ED003091EB0046
:1019F00031603093EB007093EC002093ED00509336
:101A0000F0002091EE0027FF07C09F5FD3CF8F70BB
:101A10008093E90081E0089580E008958091F201CB
:101A200087FF11C08091E80082FD05C08091F1011F
:101A30008111F8CF11C08091E8008B770BC08091A5
:101A4000F101882349F08091E80080FFF8CF809170
:101A5000E8008E778093E80008952091E4003091AB
:101A6000E50095E64091EC00842F817040FF22C094
:101A70008091E80080FD1CC08091F101882391F0E5
:101A8000853091F08091EB0085FD10C04091E4001D
:101A90005091E5004217530729F39A01915011F72D
:101AA00084E0089582E0089583E0089581E0089538
:101AB00080E008954091E80042FFDECF08950E9443
:101AC000CD0D0E94D50DE0EEF0E080818160808335
:101AD000E8EDF0E080818F77808319BCA7EDB0E05E
:101AE0008C918E7F8C9380818F7E80831092F00109
:101AF00008950F931F93CF93DF930E94CD0D0E9403
:101B0000D50DC8EDD0E088818F7788838881806883
:101B1000888388818F7D888319BC1092F10110928F
:101B2000ED011092EF011092EE0100EE10E0F801CD
:101B300080818B7F808388818160888342E060E040
:101B400080E00E94D90CE1EEF0E080818E7F8083FE
:101B5000E2EEF0E080818160808380818860808314
:101B6000F80180818E7F8083888180618883DF9106
:101B7000CF911F910F910895E8EDF0E080818F7E65
:101B80008083E7EDF0E080818160808384E082BF24
:101B900081E08093F0010C94790DE8EDF0E0808114
:101BA0008E7F80831092E20008951092DA001092E6
:101BB000E10008951F920F920FB60F9211242F93F8
:101BC0003F934F935F936F937F938F939F93AF93C5
:101BD000BF93EF93FF938091E10082FF0BC0809150
:101BE000E20082FF07C08091E1008B7F8093E100DB
:101BF0000E9441108091DA0080FF1FC08091D800C0
:101C000080FF1BC08091DA008E7F8093DA00809184
:101C1000D90080FF0DC080E189BD82E189BD09B492
:101C200000FEFDCF81E08093F1010E943C0A05C0D7
:101C300019BC1092F1010E944A0A8091E10080FFD4
:101C400019C08091E20080FF15C08091E2008E7F74
:101C50008093E2008091E20080618093E2008091B5
:101C6000D80080628093D80019BC85E08093F10190
:101C70000E944E0A8091E10084FF30C08091E20012
:101C800084FF2CC080E189BD82E189BD09B400FEDA
:101C9000FDCF8091D8008F7D8093D8008091E100A6
:101CA0008F7E8093E1008091E2008F7E8093E2003E
:101CB0008091E20081608093E2008091ED018823B1
:101CC00011F084E007C08091E30087FD02C081E04D
:101CD00001C083E08093F1010E94500A8091E100ED
:101CE00083FF29C08091E20083FF25C08091E1003D
:101CF000877F8093E10082E08093F1011092ED01F3
:101D00008091E1008E7F8093E1008091E2008E7FE0
:101D10008093E2008091E20080618093E20042E0E3
:101D200060E080E00E94D90C8091F0008860809390
:101D3000F0000E944D0AFF91EF91BF91AF919F91EA
:101D40008F917F916F915F914F913F912F910F9064
:101D50000FBE0F901F9018951F920F920FB60F9203
:101D600011242F933F934F935F936F937F938F93A0
:101D70009F93AF93BF93CF93DF93EF93FF93C09164
:101D8000E900CF708091EC00D82FD17080FDD0E8B1
:101D90001092E9008091F000877F8093F0007894A2
:101DA0000E94F00E1092E9008091F000886080930C
:101DB000F000CD2BCF70C093E900FF91EF91DF9140
:101DC000CF91BF91AF919F918F917F916F915F91D3
:101DD0004F913F912F910F900FBE0F901F9018952C
:101DE0001F93CF93DF93CDB7DEB7AA970FB6F894C2
:101DF000DEBF0FBECDBFE2EFF1E088E08E0F909125
:101E0000F10091938E13FBCF0E946C0A8091E80041
:101E100083FF1FC18091F2019091F301492F50E09F
:101E20004A30510508F015C1FA01EA5AFF4F0C94E7
:101E30002B24803881F0823809F00BC18091F601A3
:101E40008F708093E9008091EB0085FB882780F9F3
:101E50001092E90006C08091EE019091EF0191117E
:101E600082609091E800977F9093E8008093F10062
:101E70001092F100C8C0282F2D7F09F0EAC08823F6
:101E800019F0823061F0E5C08091F401813009F0F1
:101E9000E0C0933009F080E08093EF012BC0809187
:101EA000F401811127C08091F6018F7009F4D1C02F
:101EB0008093E9002091EB0020FF1CC0933021F4B7
:101EC0008091EB00806214C09091EB009061909340
:101ED000EB0021E030E0A90102C0440F551F8A95B4
:101EE000E2F74093EA001092EA008091EB008860EC
:101EF0008093EB001092E9008091E800877F86C014
:101F00008111A7C01091F4011F778091E3008078C0
:101F1000812B8093E3008091E800877F8093E80025
:101F20000E940E0D8091E80080FFFCCF8091E300BD
:101F300080688093E300111102C082E001C083E059
:101F40008093F10186C08058823008F082C0809171
:101F5000F4019091F5018C3D53E0950779F583E00C
:101F60008A838AE289834FB7F894DE01139620E0D2
:101F70003EE051E2E32FF0E050935700E49120FF60
:101F800003C0E295EF703F5FEF708E2F90E0EA3074
:101F900010F0C79601C0C0968D939D932F5F24319A
:101FA00049F74FBF8091E800877F8093E8006AE29D
:101FB00070E0CE0101960E94150C14C0AE014F5F77
:101FC0005F4F6091F6010E945C0BBC01009709F421
:101FD00040C09091E800977F9093E80089819A81B2
:101FE0000E94780C8091E8008B778093E80031C0E4
:101FF000803879F58091E800877F8093E8008091B0
:10200000ED018093F1008091E8008E778093E800E5
:102010000E940E0D1EC081111CC09091F4019230DF
:10202000C0F48091E800877F8093E8009093ED01F1
:102030000E940E0D8091ED01811106C08091E30098
:1020400087FD02C081E001C084E08093F1010E941D
:10205000580A8091E80083FF0AC08091E800877FDA
:102060008093E8008091EB0080628093EB00AA9659
:102070000FB6F894DEBF0FBECDBFDF91CF911F9199
:1020800008950895CF938091F1018823A1F0C09124
:10209000E900CF709091EC00892F817090FD80E86D
:1020A000C82B1092E9008091E80083FD0E94F00E99
:1020B000CF70C093E900CF910895909375018093FC
:1020C00074010895E0917401F0917501309721F049
:1020D0000190F081E02D099480E00895E091740171
:1020E000F0917501309721F00280F381E02D099481
:1020F0000895E0917401F0917501309721F004800A
:10210000F581E02D099408952091720130917301B9
:102110008217930771F09093730180937201E0919D
:102120007401F0917501309721F00680F781E02D60
:1021300009940895209170013091710182179307DD
:1021400071F09093710180937001E0917401F091AE
:102150007501309721F00084F185E02D09940895F0
:1021600008950C94B0100E940A1C0E948C030C94D9
:10217000CC1C9F92AF92BF92CF92DF92EF92FF92D0
:102180000F931F93CF93DF9300D000D000D0CDB733
:10219000DEB70E94A4030DE010E0AA24A394B12CA2
:1021A000902E802F0E949204980129583E4F690179
:1021B000F901F080F826A1F40150110988F78FEF9A
:1021C00089838A831B820E94131C8160782F9D83E0
:1021D0008C8349815A816B818D810E9450112FC05F
:1021E0009091DA0191FF04C08E830E9498048E8141
:1021F00025E030E0A501022E01C0440F0A94EAF761
:10220000E42E4F21C1F029839A828E2191E009F4B6
:1022100090E09B830E94131C8160782F9D838C83A8
:1022200049815A816B818D810E945011F601808114
:10223000E826E08204C021503109E0F6BDCF0E94BB
:10224000B31F109176010E9462101817B9F00E9416
:1022500062108093760126960FB6F894DEBF0FBE0B
:10226000CDBFDF91CF911F910F91FF90EF90DF9045
:10227000CF90BF90AF909F900C945B0926960FB6BD
:10228000F894DEBF0FBECDBFDF91CF911F910F91AC
:10229000FF90EF90DF90CF90BF90AF909F90089508
:1022A000CF93DF93CDB7DEB72B970FB6F894DEBF91
:1022B0000FBECDBF4F83588769877A878B87DE0132
:1022C000119686E0FD0111928A95E9F785E0FE01FD
:1022D000379601900D928A95E1F749815A816B8179
:1022E0007C818D819E810E9499172B960FB6F89460
:1022F000DEBF0FBECDBFDF91CF910895CF9388236E
:1023000009F4C2C0C82F823859F40E94621081FDBE
:10231000BBC089E30E94731A0E94401B89E30CC072
:10232000833879F40E94621080FDAEC083E50E947C
:10233000731A0E94401B83E50E94B51ACF910C943A
:10234000401B843859F40E94621082FD9DC087E4CE
:102350000E94731A0E94401B87E4EECF8CEF8C0F13
:10236000813A48F48C2F0E94F62181118DC08C2F68
:102370000E94731AE3CF80E28C0F883048F4C77054
:1023800081E001C0880FCA95EAF70E94F91AD6CFFA
:102390008BE58C0F833078F4C53A29F0C63A31F0DA
:1023A00083E890E005C081E890E002C082E890E018
:1023B000CF910C94841088E58C0F833108F064C0B1
:1023C000C83A39F1C93A41F1CA3A49F1CB3A51F127
:1023D000CC3A59F1CD3A61F1C03B69F1CE3A71F195
:1023E000CF3A79F1C13B81F1C23B89F1C33B91F115
:1023F000C43B99F1C53BA1F1C63BA9F1C73BB1F183
:10240000C83BB9F1C93BC1F1CA3BC9F180E090E0DA
:1024100038C082EE90E035C089EE90E032C08AEE9E
:1024200090E02FC085EB90E02CC086EB90E029C0B7
:1024300087EB90E026C08CEC90E023C08DEC90E020
:1024400020C083E891E01DC08AE891E01AC082E9CB
:1024500091E017C084E991E014C081E292E011C0DC
:1024600083E292E00EC084E292E00BC085E292E04B
:1024700008C086E292E005C087E292E002C08AE2EC
:1024800092E0CF910C949A10CF910895882309F48B
:102490004BC0823859F40E94621081FF45C089E325
:1024A0000E94731A0E94401B89E30CC0833871F4A8
:1024B0000E94621080FF38C083E50E94731A0E9458
:1024C000401B83E50E94B51A0C94401B843859F4D4
:1024D0000E94621082FF28C087E40E94731A0E9443
:1024E000401B87E4EFCF9CEF980F913A58F390E2AE
:1024F000980F983050F4877091E001C0990F8A9539
:10250000EAF7892F0E94FF1ADFCF9BE5980F9330DF
:1025100020F480E090E00C948410885A833120F4F9
:1025200080E090E00C949A100895882321F00E9496
:10253000F91A0C94401B0895882321F00E94FF1A79
:102540000C94401B08957F928F929F92AF92BF92FE
:10255000CF92DF92EF92FF920F931F93CF93DF936F
:102560001F92CDB7DEB77C01C62E772EFC01058108
:1025700002950F70128111110E94161B0E946C1A95
:10258000882379F0112369F080E28C0D883048F0BF
:1025900082E00E94551A0E946C1A91E0D82ED9262A
:1025A00001C0D12CE72DE295EF70F0E0E05AFF4F2B
:1025B0000C942B24872D807F072D0F70882311F01A
:1025C0000295007F112389F0002309F490C180E275
:1025D0008C0D883020F4802F0E94F91A03C0802FC0
:1025E0000E94091B0E94401B82C18C2D0E94461232
:1025F000002309F495C180E28C0D883020F4802FEF
:102600000E94FF1A03C0802F0E940F1B0E94401BD4
:1026100087C1972D907F872D8F70903211F0829512
:10262000807FCC2021F0F1E0CF16B1F01EC0112345
:1026300049F0002309F414C1013009F011C10E94CE
:10264000291B6EC1002319F0013009F469C1898387
:102650000E942C1B89810AC1112321F0023008F04D
:102660005FC1FEC001115CC101C1112321F0002333
:1026700009F4F6C03CC1002309F4F8C03EC1872D1F
:1026800086958695837090E0009719F0019761F028
:1026900047C1112321F08C2D972D937002C080E04B
:1026A00090E00E9484103CC1112321F08C2D972DC5
:1026B000937002C080E090E00E949A1031C18C2D8E
:1026C000112319F00E94BB1E02C00E94231F0E940A
:1026D000A81F26C1872D837009F052C0111120C197
:1026E0008C2D829586958770880F880F9C2D9F7002
:1026F000892E912CA12CB12C082E04C0880C991C79
:10270000AA1CBB1C0A94D2F7C4FE14C00FE010E050
:1027100020E030E0B901A80104C0440F551F661F36
:10272000771F8A95D2F7CB01BA0160957095809595
:10273000909503C060E070E0CB01272D269526958B
:10274000237030E02230310569F02330310589F003
:10275000682979298A299B292130310571F00E9445
:10276000E118DEC0682979298A299B290E94FD1871
:10277000D7C00E94E118C501B4010E94C518D0C09D
:10278000112319F0872D817001C08695882309F4E3
:10279000C7C08C2D829586958770880F880F9C2DD9
:1027A0009F70892E912CA12CB12C082E04C0880C6E
:1027B000991CAA1CBB1C0A94D2F7C4FE14C00FE0DB
:1027C00010E020E030E0B901A80104C0440F551F1B
:1027D000661F771F8A95D2F7CB01BA016095709575
:1027E0008095909503C060E070E0CB01272D269581
:1027F00026952370422F50E04230510569F0433056
:10280000510589F0682979298A299B294130510588
:1028100071F00E94BB1984C0682979298A299B29F3
:102820000E94D7197DC00E94BB19C501B4010E9446
:102830009F1976C08C2D90E0FC01E05EF109E53136
:10284000F10508F050C0E059FF4F0C942B240C2DDB
:102850000F70872D8F71112331F00E943819802F4E
:102860000E9495125DC00E945919802F0E949C12EF
:1028700057C0112339F0011153C0872D8F710E9469
:102880007E194EC0023008F04BC0F7CF112339F04B
:10289000872D8F710E94381943C01123C9F3872DEA
:1028A0008F710E9459193CC0112329F0872D8F7117
:1028B0000E94231935C00E94191932C0112351F00A
:1028C000172D1F71812F0E94381963E0812F0E94FC
:1028D0004C1A26C081E00E94551A023008F182E0AD
:1028E0000E94551A1DC0112331F0002389F28C2D4E
:1028F0000E947E1115C0002391F28C2D0E94461279
:102900000FC0472D4F706C2DC7010E946E050E94AD
:102910003D1806C0472D4F706C2DC7010E946A06F6
:10292000DD20F9F00E94481A80FD1BC0F7011282D9
:102930000E94421A0E943819C7010E94C0140E94C6
:10294000421A0F90DF91CF911F910F91FF90EF905E
:10295000DF90CF90BF90AF909F908F907F900C941E
:1029600059190F90DF91CF911F910F91FF90EF9028
:10297000DF90CF90BF90AF909F908F907F90089501
:102980000F931F93CF93DF93EC01888199812B8163
:102990003C81232BB9F09F3F11F48F3F99F0CE017A
:1029A0000E94C205882371F0688179818A810E9422
:1029B0003E1A8C010E94F3190E94BA18B801CE0188
:1029C0000E94A312DF91CF911F910F9108950E9451
:1029D000161B0E94261B0E94EB1A0E94401B0E949D
:1029E00059200E94A81F80E090E00E94841080E09F
:1029F00090E00C949A100E94061B0C94E7140E941D
:102A0000331A292F22952F7030E02C3031054CF4E9
:102A10002A3031056CF42250310922303105A8F4F6
:102A200007C02C30310569F02F30310551F00DC051
:102A3000803F69F018F4803E40F409C0843F29F4D7
:102A400006C093FB882780F9089580E0089581E00F
:102A50000895CF93DF9300D000D01F92CDB7DEB79B
:102A60000F900F900F900F900F90DF91CF910895DE
:102A7000CF93DF9300D000D000D0CDB7DEB726963D
:102A80000FB6F894DEBF0FBECDBFDF91CF91089592
:102A90001F93CF93DF93C091850116E0809186014B
:102AA000C81799F0D0E01C9FF0011D9FF00D112474
:102AB000E957FE4F40815181628173818481958104
:102AC0000E9438152196C770E9CFDF91CF911F91F1
:102AD00008954091B7015091B8016091B90170918A
:102AE000BA018091BB019091BC010C943815809182
:102AF000BC0182958F7009F054C08091B901882380
:102B000009F44FC080918501A09186016091B701C1
:102B10007091B8014091BA015091BB01B6E08A179B
:102B200009F43FC090E041155105C1F17F3F11F418
:102B30006F3FA1F1B89FF001B99FF00D1124E95743
:102B4000FE4F218172132AC02081621327C0228187
:102B5000211124C0238134812417350710F421501A
:102B60003109241B350B283C3105C0F42091BC01F0
:102B70002F7020612093BC0126E0289FF001299F3F
:102B8000F00D1124E457FE4F80818F7080618083A7
:102B900087EB91E00E94C0140C9448150196877051
:102BA000BECF0895CF92DF92EF92FF920F931F93C3
:102BB000CF93DF93CDB7DEB762970FB6F894DEBF41
:102BC0000FBECDBF8C0185E0F801DE011D9601909E
:102BD0000D928A95E1F7D8014C9111965C9111976D
:102BE00012966C9112971396CD90DC9014973091B9
:102BF000B7017091B8018091BA019091BB01009723
:102C000009F46BC17F3F19F43F3F09F466C1E090BE
:102C1000B901EE2009F4C0C02091BC01C816D90644
:102C200028F0F601E81BF90BCF0104C080959095C0
:102C30008C0D9D1DFF24F394883C910578F0F12CB8
:102C4000207F09F0C6C07C2DD98AC88A89890E9454
:102C5000291587EB91E00E94C014B1C0822F807FBC
:102C600009F046C0751314C0341312C0611110C0AE
:102C70002F7020612093BC010E94691587EB91E0C1
:102C80000E94C0148091BC01D80115968C932EC06F
:102C9000CD2819F15F3F11F44F3FF9F0F62E611185
:102CA0001CC0809185012091860136E0821709F4CD
:102CB0005AC090E0389FF001399FF00D1124E95778
:102CC000FE4F7181571306C07081471303C0728194
:102CD000711103C001968770E9CFF62E662309F4BF
:102CE00018C18091BC0181608093BC01F12C11C19D
:102CF000751308C0341306C0611104C08091BC0173
:102D0000D801C3C04D875E878D859E856A8B0E94E2
:102D1000FF146A898823E1F16623D1F12091BC0177
:102D2000822F82958F7090E0029774F08091B701A6
:102D30009091B80198878F831986DB86CA862C8785
:102D4000CE0107960E94C01486E0F801A7EBB1E01F
:102D500001900D928A95E1F70E9477150E946915FE
:102D6000FF24F394D6C04D875E878D859E850E9493
:102D7000331A292F22952F7030E0223031050CF0C4
:102D8000BCC09F7009F0B6C0805E883008F4C1C036
:102D9000C8010E94C014E4CFC816D90608F453C075
:102DA000F601E81BF90BCF01883C910508F450C0EF
:102DB000F12C7C2DD98AC88A89890E942915E7EBD4
:102DC000F1E086E0DF011D928A95E9F70E9469151E
:102DD000A0C0751314C0341312C0611110C08091CB
:102DE000BC01F8018583C8010E94C01486E0E7EBAE
:102DF000F1E0DF011D928A95E9F7FE2C8AC04D872C
:102E00005E878D859E856A8B0E94FF146A89882360
:102E100009F4BECF662309F4BBCF2091BC01822FF9
:102E200082958F7090E002970CF48ECF8091B7015D
:102E30009091B8019A8389831B82DD82CC822E8394
:102E4000CE0101967FCF809590958C0D9D1DACCFC6
:102E5000F62E662309F49CCF75132EC034132CC0B4
:102E60002091BC0120FD1FC0822F82958F70D9F068
:102E7000D80115962C9315978F3049F08F5F982FB6
:102E80009295907F822F8F70892B15968C93C80115
:102E90000E94C01486E0F801A7EBB1E001900D920A
:102EA0008A95E1F793CF86E0F801A7EBB1E00190B6
:102EB0000D928A95E1F72DC04D875E878D859E85A1
:102EC0000E94FF14811140CF8091BC0181608093EA
:102ED000BC01C8010E94C0141CC0662309F458CF6D
:102EE0004D875E878D859E850E94FF14882309F497
:102EF0004FCF2ACF811148CF0CC0243031050CF0C0
:102F000047CF9F7009F440CFF8019581907F09F079
:102F10003BCF8F2D62960FB6F894DEBF0FBECDBFAC
:102F2000DF91CF911F910F91FF90EF90DF90CF90A5
:102F300008951F93CF93DF93CDB7DEB72C970FB6CD
:102F4000F894DEBF0FBECDBF4F83588769877A875D
:102F50008B879C87CE0107960E94D215882369F043
:102F60008F8198852A853B85232BF1F19F3F09F0BE
:102F700063C08F3F09F060C037C086E0FE0137961E
:102F8000DE01119601900D928A95E1F76F817885A7
:102F9000EA85FB85309741F17F3F11F46F3F21F1C6
:102FA0002091860130E0C9010196877099274091F0
:102FB000850150E08417950709F447C069837A8337
:102FC000FD83EC8396E0929FD001939FB00D112476
:102FD000A957BE4FFE01319601900D929A95E1F7E7
:102FE000809386010E94481516E08091850190919A
:102FF00086018917C1F1189FC001112489579E4F7E
:103000000E94D215882379F1E09185011E9FF0017D
:103010001124E957FE4F408151816281738184817F
:1030200095810E9438158091850190E00196877006
:10303000992780938501D9CF4F81588569857A85F5
:103040008B859C850E943815CFCF0E94FB1410926F
:10305000860110928501E7EBF1E086E0DF011D9229
:103060008A95E9F7C1CF2C960FB6F894DEBF0FBE54
:10307000CDBFDF91CF911F910895EF92FF920F93F3
:103080001F93CF93DF938C01009709F46CC0F12C50
:10309000EE24E394E8012196F8018491843740F40A
:1030A000843008F051C0813081F0823019F15BC06A
:1030B000853709F444C0A8F19CE7980F903708F0D1
:1030C00052C08F770E94461241C00E5F1F4FFE0113
:1030D000C49180E28C0F883048F4C7708E2D01C0F7
:1030E000880FCA95EAF70E94191B14C08C2F0E9402
:1030F0007E112DC00E5F1F4FFE01C49180E28C0F28
:10310000883058F4C7708E2D01C0880FCA95EAF731
:103110000E941F1B0E94401B1AC08C2F0E94461247
:1031200016C00E5F1F4FFE01C491CC2381F08FE9C2
:103130009FE00197F1F700C00000C150F6CF0E5F8D
:103140001F4FFE01F49003C00E947E118E018F2D4F
:10315000882309F49FCFEFE9FFE03197F1F700C032
:1031600000008150F5CFDF91CF911F910F91FF901B
:10317000EF90089508956093C1017093C201809308
:10318000C3019093C4010C94E7140F931F93009113
:10319000C1011091C2012091C3013091C401DC0131
:1031A000CB01802B912BA22BB32B8093C101909349
:1031B000C201A093C301B093C4011F910F910C945D
:1031C000E7140F931F930091C1011091C201209148
:1031D000C3013091C401DC01CB0180239123A223E0
:1031E000B3238093C1019093C201A093C301B09314
:1031F000C4011F910F910C94E7140F931F9300913A
:10320000C1011091C2012091C3013091C401DC01C0
:10321000CB0180279127A227B3278093C1019093E8
:10322000C201A093C301B093C4011F910F910C94EC
:10323000E7141092BD011092BE011092BF011092CE
:10324000C0010C94E71441E050E060E070E004C07D
:10325000440F551F661F771F8A95D2F74093BD0113
:103260005093BE016093BF017093C0010C94E714AA
:1032700041E050E060E070E004C0440F551F661F5D
:10328000771F8A95D2F78091BD019091BE01A091E0
:10329000BF01B091C001482B592B6A2B7B2B409367
:1032A000BD015093BE016093BF017093C0010C94A7
:1032B000E71441E050E060E070E004C0440F551FA7
:1032C000661F771F8A95D2F7409550956095709547
:1032D0008091BD019091BE01A091BF01B091C0014C
:1032E000482359236A237B234093BD015093BE0199
:1032F0006093BF017093C0010C94E71441E050E06B
:1033000060E070E004C0440F551F661F771F8A9568
:10331000D2F78091BD019091BE01A091BF01B09103
:10332000C001482759276A277B274093BD01509346
:10333000BE016093BF017093C0010C94E7140F931A
:103340001F930091BD011091BE012091BF013091EA
:10335000C001DC01CB01802B912BA22BB32B8093DE
:10336000BD019093BE01A093BF01B093C0011F9116
:103370000F910C94E7140F931F930091BD011091CE
:10338000BE012091BF013091C001DC01CB0180233F
:103390009123A223B3238093BD019093BE01A093F8
:1033A000BF01B093C0011F910F910C94E7140F93CC
:1033B0001F930091BD011091BE012091BF0130917A
:1033C000C001DC01CB0180279127A227B32780937E
:1033D000BD019093BE01A093BF01B093C0011F91A6
:1033E0000F910C94E7140895CF92DF92EF92FF9221
:1033F0000F931F93CF93DF938C01C090C101D090A6
:10340000C201E090C301F090C4018091BD01909190
:10341000BE01A091BF01B091C001C82AD92AEA2AF1
:10342000FB2ACFE1D0E0D701C6010C2E04C0B6952F
:10343000A795979587950A94D2F780FF06C0B801A3
:103440008C2F0E94C008019721F4219760F780E03B
:1034500001C08C2FDF91CF911F910F91FF90EF90C2
:10346000DF90CF900895CF93DF93EC010E94F41981
:10347000BE010E94C008DF91CF910895CB010E9448
:10348000331A08958091C501859585958595089590
:103490008091C5018770089598E0899F900111245B
:1034A000262B2093C5010C9438192091C5018095D5
:1034B00082238093C501982F977069F430E0482FDC
:1034C000552747FD50952417350729F08595859593
:1034D00085950C94591908959091C501977081E0D4
:1034E00009F480E0089590910C01992321F09091C6
:1034F0000D01911109C020910E0130910F01F901C8
:1035000032969FEF40E01FC0982F9695969596951E
:103510009F3050F5E0910E01F0910F01E90FF11D80
:10352000877021E030E0A90102C0440F551F8A9541
:10353000E2F7CA019181892B818308959F3F39F079
:103540004F5F4E3041F051915813F8CF0DC05111DB
:10355000F7CF942FF5CF9F3F39F0F901E90FF11D17
:1035600097FDFA9582830895089590910C0199230F
:1035700021F090910D01911109C020910E0130911F
:103580000F01F9013296205F3F4F1FC0982F96958B
:10359000969596959F30F0F4E0910E01F0910F0111
:1035A000E90FF11D877021E030E0A90102C0440F4E
:1035B000551F8A95E2F7CA018095918189238183FD
:1035C00008953196E217F30729F090819813F9CF07
:1035D0001082F7CF089581E090E0E0910E01F09124
:1035E0000F01E80FF91F1082019680319105A9F7AC
:1035F00008959091D901892B8093D90108958095E0
:103600009091D90189238093D90108951092D9010D
:1036100008959091D801892B8093D80108958095C1
:103620009091D80189238093D80108951092D801F0
:1036300008959091D701892B8093D70108958095A3
:103640009091D70189238093D70108951092D701D3
:1036500008958093C60108951092C601089580913F
:103660000E0190910F01FC0131969C01205F3F4FAC
:1036700080E0919191118F5FE217F307D1F70895E0
:10368000E0910E01F0910F018091D9018083E091CA
:103690000E01F0910F0190818091D801892B8083D8
:1036A000E0910E01F0910F0190818091D701892B5B
:1036B00080838091C601882361F0E0910E01F09132
:1036C0000F019081892B80830E942F1B8111109202
:1036D000C60180910E0190910F010C946E1020E0B4
:1036E000009739F0AC0141505109842395232F5F95
:1036F000F7CF822F0895CF92DF92EF92FF926C0165
:10370000EE24FF24C114D104E104F10421F0C70127
:10371000B60120E101C020E0C72ED82EE92EFF24FB
:10372000C114D104E104F10419F0285FC701B60106
:103730006B017C0154E0F694E794D794C7945A95B2
:10374000D1F7C114D104E104F10419F02C5FC701D1
:10375000B6016B017C0142E0F694E794D794C794DC
:103760004A95D1F7C114D104E104F10419F02E5F98
:10377000C701B601DC01CB01B695A7959795879552
:10378000892B8A2B8B2B09F02F5F822FFF90EF90D4
:10379000DF90CF9008958091F101843021F1109253
:1037A000DB0120E488E190E00FB6F894A8958093BF
:1037B00060000FBE2093600080E00E945B0983B729
:1037C000817F846083BF83B7816083BF789488954D
:1037D00083B78E7F83BF88E10FB6F8948093600033
:1037E000109260000FBE0895089508950E94F41B82
:1037F0000E94A4030E94F51B0E94990491E081118C
:1038000001C090E0892F08950E94FB140E9462106D
:103810000C945B0982E084BD93E095BD9AEF97BD5F
:1038200080936E0008952FB7F8948091DC019091F9
:10383000DD01A091DE01B091DF012FBF0895CF928D
:10384000DF92EF92FF920F931F932FB7F89440915E
:10385000DC015091DD016091DE017091DF012FBF2D
:103860006A017B01EE24FF248C0120E030E0C016C9
:10387000D106E206F30610F4415051099A01281BC3
:10388000390BC9011F910F91FF90EF90DF90CF90FE
:1038900008951F920F920FB60F9211248F939F934A
:1038A000AF93BF938091DC019091DD01A091DE0187
:1038B000B091DF010196A11DB11D8093DC019093B1
:1038C000DD01A093DE01B093DF01BF91AF919F9125
:1038D0008F910F900FBE0F901F9018950E945F0D53
:1038E000F8942FEF87EA91E6215080409040E1F76D
:1038F00000C0000087E090EBDC018093FB01909317
:10390000FC01A093FD01B093FE019CE088E10FB69D
:10391000F894A895809360000FBE90936000FFCF4D
:10392000EF92FF920F931F93CF93DF93D82FCDE0A9
:103930008C2F0E94920405E010E0E82EF12CC701C4
:10394000002E02C0959587950A94E2F780FF09C082
:10395000602F7C2F80E00E946B06D81302C081E0AC
:1039600006C00150110958F7C15010F780E0DF91EF
:10397000CF911F910F91FF90EF900895CF93C82F93
:103980008CE20E94901C882321F08C2FCF910C9404
:10399000901C80E0CF910895CF930E94131E811157
:1039A00002C00E94F91DC5E6C15049F00E94A4035F
:1039B0008FE39CE90197F1F700C00000F5CF89E2A1
:1039C0000E94BE1C811113C18AE20E94BE1C81119B
:1039D0000E94F91D85E00E94BE1C81110E946E1C90
:1039E0000E941E1E8093DA0187E00E94BE1C88237D
:1039F000A9F18BE10E94BE1C882351F08091DA016D
:103A000081FB222720F991E0922790FB81F90EC0DB
:103A10008EE00E94BE1C882361F08091DA0182FB57
:103A2000222720F991E0922790FB82F98093DA0116
:103A300015C080E10E94BE1C9091DA01882341F0FC
:103A400093FB222720F981E0822780FB93F904C0B1
:103A5000892F809580FB90F99093DA018091DA01AB
:103A60000E94221E0E94301E8093FA0180EE0E9466
:103A7000BE1C882341F08091FA01982F909590FB0D
:103A800080F98093FA0189E30E94BE1C882359F0D3
:103A90008091FA0181FB222720F991E0922790FB87
:103AA00081F98093FA0182EE0E94BE1C882359F0AE
:103AB0008091FA0182FB222720F991E0922790FB66
:103AC00082F98093FA0186EE0E94BE1C882359F089
:103AD0008091FA0183FB222720F991E0922790FB45
:103AE00083F98093FA0183EE0E94BE1C882359F06B
:103AF0008091FA0184FB222720F991E0922790FB24
:103B000084F98093FA0185E30E94BE1C882359F052
:103B10008091FA0185FB222720F991E0922790FB02
:103B200085F98093FA0181E30E94BE1C882359F035
:103B30008091FA0186FB222720F991E0922790FBE1
:103B400086F98093FA0181E10E94BE1C882359F016
:103B50008091FA0187FB222720F991E0922790FBC0
:103B600087F98093FA018091FA010E94341E8091B6
:103B7000FA0187FB882780F980930D0187E20E9474
:103B8000BE1CC82F8EE10E94BE1C8111C2608FE155
:103B90000E94BE1C8111C46080E20E94BE1C811183
:103BA000C86081E20E94BE1C8111C06182E20E9455
:103BB000BE1C8111C06283E20E94BE1C8111C064E0
:103BC00084E20E94BE1C882311F0C06802C0CC238E
:103BD00029F08C2F0E942B1E6C2F03C00E94271EE1
:103BE000682F70E080E090E0CF910C94BB18CF91EB
:103BF00008956DEE7EEF80E090E00E94652460E025
:103C000082E090E00E94532460E083E090E00E9414
:103C1000532460E084E090E00E94532460E085E05B
:103C200090E00C94532480E090E00E944D2421E029
:103C30008D3E9E4F09F020E0822F089582E090E0B3
:103C40000C944524682F82E090E00C94532483E088
:103C500090E00C944524682F83E090E00C9453246A
:103C600084E090E00C944524682F84E090E00C946C
:103C700053248091E20180FF0BC06091130185E025
:103C8000689FB001112475956795759567952BC050
:103C900081FF09C06091130185E0689FB001112484
:103CA0007595679520C082FF07C06091130185E07C
:103CB000689FB001112417C09091E3019923D1F0BE
:103CC00060911201961788F72091130185E0289FD3
:103CD00090011124929FA001939F500D112470E038
:103CE000CA010E9417246038710540F461157105FE
:103CF00039F002C065E070E0862F08958FE70895DF
:103D000081E008958091E20180FF08C06091110177
:103D100070E0759567957595679521C081FF06C020
:103D20006091110170E07595679519C082FF04C01C
:103D30006091110170E010C09091E3019923C1F0EE
:103D4000609110019617A0F780911101899FC00121
:103D5000112470E00E9417246038710528F4611561
:103D6000710521F0862F08958FE7089581E0089569
:103D700061E070E0F4CF803F21F40E94391E81950C
:103D800004C0813F29F40E94391E8093E601089502
:103D9000823F21F40E94391E819504C0833F29F49B
:103DA0000E94391E8093E5010895893F19F40E940D
:103DB000821E05C08A3F31F40E94821E8195809345
:103DC000E70108958B3F21F40E94821E819504C073
:103DD0008C3F29F40E94821E8093E8010895843F5D
:103DE00021F48091E401816017C0853F21F4809126
:103DF000E401826011C0863F21F48091E401846077
:103E00000BC0873F21F48091E401886005C0883FA2
:103E100031F48091E40180618093E40108958D3F45
:103E200021F48091E20181600BC08E3F21F48091EA
:103E3000E201826005C08F3F29F48091E201846035
:103E40008093E2010895803F39F48091E60187FF75
:103E50006CC01092E60169C0813F29F48091E601AF
:103E60001816BCF362C09091E501823F29F497FFD8
:103E70005CC01092E50159C0833F19F41916CCF3C8
:103E800054C0893F41F48091E70118160CF04DC0F1
:103E90001092E7014AC08A3F29F48091E70187FF29
:103EA00044C0F6CF8B3F39F48091E80187FF3DC0D5
:103EB0001092E8013AC08C3F29F48091E80118166D
:103EC000BCF333C0843F21F48091E4018E7F17C09E
:103ED000853F21F48091E4018D7F11C0863F21F45C
:103EE0008091E4018B7F0BC0873F21F48091E40136
:103EF000877F05C0883F31F48091E4018F7E8093F5
:103F0000E40113C08D3F21F48091E2018E7F0BC04C
:103F10008E3F21F48091E2018D7F05C08F3F29F40F
:103F20008091E2018B7F8093E2018091E501811114
:103F30000EC08091E60181110AC08091E7018111D4
:103F400006C08091E801811102C01092E30108953A
:103F500084EE91E00E9479100E94131C9093E1017D
:103F60008093E00108951F93CF93DF938091E00148
:103F70009091E1010E941F1CAC019091E3019923F3
:103F800021F02091140130E006C0209115018AE053
:103F9000289F900111244217530708F486C080918E
:103FA000E501C091E601D091E7011091E80181118E
:103FB00007C0C11176C0D11174C0111172C075C093
:103FC0009F3F19F09F5F9093E301181624F40E941D
:103FD000391E8093E5018091E50187FF05C00E94AD
:103FE000391E81958093E5011C1624F40E94391E28
:103FF0008093E6018091E60187FF05C00E94391E8B
:1040000081958093E6016091E501662339F1C091C5
:10401000E601CC2319F1772767FD7095872F972F3D
:104020000E94282323E333E343E35FE30E948C23CE
:104030000E94F5226093E5016C2F772767FD70954C
:10404000872F972F0E94282323E333E343E35FE383
:104050000E948C230E94F5226093E6011D1624F431
:104060000E94821E8093E7018091E70187FF05C0CF
:104070000E94821E81958093E701111624F40E940C
:10408000821E8093E8018091E80187FF05C00E94AD
:10409000821E81958093E801DF91CF911F910C944E
:1040A000A81F9F3F09F08ECF96CFDF91CF911F9130
:1040B0000895E4EEF1E085E0DF011D928A95E9F7CD
:1040C0001092E3011092E2010895833081F128F407
:1040D000813059F08230D1F00895853009F449C01B
:1040E000B8F1863009F456C0089580911501262F45
:1040F00030E0280F311D2F3F310524F4680F609305
:10410000150108958FEF8093150108958091140192
:10411000262F30E0280F311D2F3F310524F4680F82
:104120006093140108958FEF809314010895809196
:104130001301262F30E0280F311D2F3F310524F4C5
:10414000680F6093130108958FEF80931301089512
:1041500080911201262F30E0280F311D2F3F3105AD
:1041600024F4680F6093120108958FEF8093120179
:10417000089580911101262F30E0280F311D2F3F27
:10418000310524F4680F6093110108958FEF809337
:104190001101089580911001262F30E0280F311D64
:1041A0002F3F310524F4680F6093100108958FEFBD
:1041B000809310010895833011F128F4813049F083
:1041C000823091F00895853081F120F18630C1F17F
:1041D000089580911501681720F4861B80931501BE
:1041E000089510921501089580911401681720F424
:1041F000861B8093140108951092140108958091F4
:104200001301681720F4861B809313010895109200
:104210001301089580911201681720F4861B809382
:1042200012010895109212010895809111016817EA
:1042300020F4861B809311010895109211010895B6
:1042400080911001681720F4861B80931001089557
:104250001092100108950F931F938D3109F46BC0D4
:1042600008F03FC08E3009F47FC0C0F4873009F4F5
:1042700069C068F4863009F0B1C08091DA01817FAD
:104280008E7F8093DA0181E08093EA01A8C08830B4
:1042900009F4A2C08B3009F49FC0A0C0863109F494
:1042A0009BC078F4803109F472C0813109F096C066
:1042B0000E94FB1490910D0181E0892780930D01EC
:1042C0008BC0893109F488C08B3109F087C0809197
:1042D000DA0181FB222720F991E0922790FB81F9F6
:1042E0004CC0853309F470C048F4873209F46CC0BF
:1042F00008F459C0893209F467C070C0833438F4B7
:104300008A3308F04EC0883309F466C067C083342E
:1043100009F45AC0883409F061C00E94FB140FEF01
:1043200013ED20E3015010402040E1F700C00000F1
:104330000E946E1C51C00E94AF220E9462100E9417
:104340005B094AC09091DA01892F8095817080FBCA
:1043500090F929F0966098609093DA0140C0997FB7
:10436000977F9093DA0138C08091DA0182FB22278F
:1043700020F991E0922790FB82F98093DA0199234A
:1043800059F18091DA0181608093DA0125C0809132
:10439000DA0183FB222720F991E0922790FB83F931
:1043A000ECCF895301C08D5141E050E060E070E0F6
:1043B0008A019B0104C0000F111F221F331F8A9521
:1043C000D2F7C901B80104C061E070E080E090E07C
:1043D0000E94BB180E94FB1481E001C080E01F9185
:1043E0000F91089580E0089580E00895CF93C82F3D
:1043F0008091EA01813079F018F08230E9F187C0CC
:10440000E0910E01F0910F018081813169F08232DB
:1044100009F07FC009C0E0910E01F0910F01808189
:10442000813111F0823261F48C2F0E94F2218111CE
:1044300004C08C2F0E942B211DC081E090E01AC087
:104440008C2F0E94F421811114C0C43179F048F4FA
:10445000CB3079F0C03109F060C082E08093EA018E
:1044600008C0C93219F0C83321F057C01092EA01D0
:1044700054C081E0817053C0C93289F118F5C4314C
:1044800071F1A8F4C73009F046C08AE080931501A5
:1044900094E19093140193E090931301809312019F
:1044A00088E08093110188E28093100134C0CE51DE
:1044B000C63088F5EC2FF0E0E65DFE4F80818093FA
:1044C000E90129C0CE34E9F020F4CB3421F56AE0CB
:1044D00013C0C13579F0C235F1F461E00DC08091AF
:1044E000E901882319F01092E90115C081E0809359
:1044F000EA0115C061E006C08091E9010E946520D3
:104500000AC06AE08091E9010E94DB2004C0109299
:10451000EA0180E004C081E002C080E0ABCFCF912F
:104520000895E1E8F0E08081886080838081816087
:1045300080838FB7F89493E09093890090ED9093E7
:1045400088008FBF0895EFE6F0E08081826080836D
:104550000895EFE6F0E080818D7F80830895EFE697
:10456000F0E0908182E08927808308951F920F9266
:104570000FB60F9211242F933F934F935F936F9336
:104580007F938F939F93AF93BF93EF93FF9380910C
:10459000EB019091EC0101969093EC018093EB017B
:1045A000811103C082E00E945B09E091EC01E69575
:1045B000E695F0E0EB59FA4FE4918091EB018E1310
:1045C00003C080E00E945B09FF91EF91BF91AF9122
:1045D0009F918F917F916F915F914F913F912F911B
:1045E0000F900FBE0F901F90189504D06894B111D2
:1045F0008DC0089570D088F09F5790F0B92F9927FB
:10460000B751A0F0D1F0660F771F881F991F1AF0DD
:10461000BA95C9F712C0B13081F077D0B1E00895F2
:1046200074C0672F782F8827B85F39F0B93FCCF373
:10463000869577956795B395D9F73EF490958095D3
:10464000709561957F4F8F4F9F4F0895E89409C0F3
:1046500097FB3EF490958095709561957F4F8F4FB5
:104660009F4F9923A9F0F92F96E9BB279395F695CB
:10467000879577956795B795F111F8CFFAF4BB0F49
:1046800011F460FF1BC06F5F7F4F8F4F9F4F16C0AD
:10469000882311F096E911C0772321F09EE8872F37
:1046A000762F05C0662371F096E8862F70E060E0F3
:1046B0002AF09A95660F771F881FDAF7880F96956C
:1046C000879597F9089557FD9058440F551F59F055
:1046D0005F3F71F04795880F97FB991F61F09F3FEF
:1046E00079F087950895121613061406551FF2CF18
:1046F0004695F1DF08C0161617061806991FF1CF68
:1047000086957105610508940895E894BB2766278E
:104710007727CB0197F908950BD078C069D028F09E
:104720006ED018F0952309F05AC05FC01124EECF67
:10473000CADFA0F3959FD1F3950F50E0551F629FFC
:10474000F001729FBB27F00DB11D639FAA27F00DEA
:10475000B11DAA1F649F6627B00DA11D661F829F11
:104760002227B00DA11D621F739FB00DA11D621FF6
:10477000839FA00D611D221F749F3327A00D611D13
:10478000231F849F600D211D822F762F6A2F1124F5
:104790009F5750408AF0E1F088234AF0EE0FFF1F48
:1047A000BB1F661F771F881F91505040A9F79E3F7F
:1047B000510570F014C0AACF5F3FECF3983EDCF3D4
:1047C000869577956795B795F795E7959F5FC1F7BC
:1047D000FE2B880F911D9695879597F9089597F967
:1047E0009F6780E870E060E008959FEF80EC089597
:1047F00000240A94161617061806090608950024C0
:104800000A9412161306140605060895092E039439
:10481000000C11F4882352F0BB0F40F4BF2B11F4AD
:1048200060FF04C06F5F7F4F8F4F9F4F089597FBCE
:10483000072E16F4009407D077FD09D00E9431248A
:1048400007FC05D03EF4909581959F4F0895709593
:1048500061957F4F0895EE0FFF1F0590F491E02DB5
:104860000994AA1BBB1B51E107C0AA1FBB1FA617B7
:10487000B70710F0A61BB70B881F991F5A95A9F709
:1048800080959095BC01CD010895F999FECF92BD18
:1048900081BDF89A992780B50895A8E1B0E042E07B
:1048A00050E00C946D24262FF999FECF92BD81BD66
:1048B000F89A019700B4021639F01FBA20BD0FB65E
:1048C000F894FA9AF99A0FBE08950196272F0E943C
:1048D00054240C945324DC01CB01FC01F999FECF44
:1048E00006C0F2BDE1BDF89A319600B40D92415078
:0A48F0005040B8F70895F894FFCF88
:1048FA0002205D09EB09C809940960090101C70191
:10490A0028080A03140A3F4D36392605D904A30498
:10491A006A04FD0316042F04480401020304050671
:04492A000708090071
:00000001FF
